:020000020000FC
:100000005DCD9BC1000000001FC0000088C0000043
:10001000000092C00000000000000000020304067F
:10002000080C10182030406080000406080C1018DE
:100030002030406080A0C0000003070F1F000505AE
:100040000D050205030302004FB662FD0CC05520EA
:1000500041F00994C52DC095089483FDC795C4BD92
:1000600064604FBE1895C0916400089483FDC795E5
:10007000C4BD6B7FC0916400CF3F09F419C04FBE6F
:10008000909891989398189590989198939876FD58
:100090000DC064FD0BC0C9E0CA95F1F7C091B10075
:1000A000C0FD959AC1FD979AC2FD949A4FBE1895CE
:1000B00024BCCC27C064C8BF6460F8CFCBCF70FF2E
:1000C000C9CF64FDC7CF909AC5CF70FFC3CF64FD81
:1000D000C1CF919ABFCF70FFBDCF64FDBBCF939AC4
:1000E000B9CF959870FFB6CF64FDB4CFCEE1CA9575
:1000F000F1F7909AAFCF979870FFACCF64FDAACF7D
:10010000CEE1CA95F1F7919AA5CF949870FFA2CF4E
:1001100064FDA0CFCEE1CA95F1F7939A9BCF4FB67D
:10012000C9B7CF7EC9BF6E7FCCB5CE0DDDB5DF1DA3
:10013000DBBDCABD4FBE18953FB68F7EABB7A0746E
:10014000A2118061A0E0ABBFA9B7AE7FA9BF789430
:10015000A0916800AA2341F085FD2EC0A0916800FF
:10016000AA95A093680028C040E050E085FD14C027
:10017000A0B396FDA095A2FD4FEFA3E096FDA2E0EF
:10018000A5BFAA27A064AABF8D7FA0B396FDA095A6
:10019000A2FD5FEF451741F7A8E161FDA09368005C
:1001A00085FD03C0A8E1A09368004093960081609C
:1001B000442311F02092990085FD0EC0A0916900A2
:1001C000AA2331F0A0916900AA95A093690004C008
:1001D0008061AA27A064AABF80FF3DC0A0919600BD
:1001E0004A2F61FF8E7F85FD18C0403F08F040EF29
:1001F000A42FA295AF704A0F5091B600533069F00A
:10020000A695A69550FD01C0A69552FD03C0A41B5E
:100210004A2F03C04A0F08F44FEFA0919F004A17DE
:1002200008F44A2F40936100A72FA670A1F073FD38
:1002300012C0A0917000AA0FAA0F50919E0056956F
:100240005695541708F0452F4A0F4093610018F453
:10025000AFEFA0936100A0916100A0936300409173
:100260006300A0919B004A1708F04A2F542EA091DA
:10027000A000AA2309F422C0542F5A1B10F4A42F63
:1002800050E0BA2E8894AA1FAA2EA091A200A09591
:10029000AA22A50E58F0A091A100A21509F0AA95D6
:1002A000AA0EA093A10048F04A2D08C0A091A10079
:1002B000BA1608F0A395A093A1004FEF40936400F5
:1002C000A0916000A395A093600051F0F894A9B7A5
:1002D000A160A9BF84FF02C0A0E4ABBF3FBE1895D8
:1002E000A0917400A395A093740041E05091680020
:1002F000552329F085FF03C05A9550936800A091BB
:100300009600A13018F0209299000DC020929A001A
:100310002092A300A0919900AF5FA093990018F0DC
:10032000AFEFA0939900F894A9B7A160A9BF84FF8B
:1003300002C0A0E4ABBF3FBE18953FB64CB55DB55B
:100340008F7EABB7A074A2118061A0E0ABBFA9B74C
:10035000AE7FA9BF789481FD23C0A2E096FDA3E003
:10036000A5BF8260A0B396FDA095A2FF05C04093F3
:100370006500509366003EC1A3E096FDA2E0A5BFD4
:10038000AA27A064AABF8D7F85FF01C026C140E0D7
:10039000A0B396FDA095A2FD20C1409396000FC189
:1003A000A3E096FDA2E0A5BF8D7F61FF71C0A2E032
:1003B00096FDA3E0A5BFAA27A064AABF82604093D0
:1003C000910050939200A0908F004A19B090900035
:1003D0005B09BB24A22C4C38520518F420929500DE
:1003E00049C0A091D400AA2359F1483C520528F4F1
:1003F000A0E1BA2EAAE0AA2E23C04836A1E05A07EF
:1004000028F4A8E0BA2EAFE0AA2E1AC0403DA2E020
:100410005A0728F4A4E0BA2EAEE1AA2E11C0403A41
:10042000A5E05A0728F4A2E0BA2EACE3AA2E08C031
:100430004839A8E05A0720F4A1E0BA2EA8E7AA2E6E
:10044000C42EA0919300CA1AD52EA0919400DA0A66
:10045000DD202AF4AFEFC094D094CA1ADA0A2092B1
:100460009500A8E0A210A0E0CA14DA0618F4A1E0F2
:10047000A093950040939300509394004091910075
:100480005091920040938F005093900042E097C0AB
:10049000A09165004A1BA09166005A0B94FD82C092
:1004A00093FD80C092FD7CC086FF03C0D52EC42E74
:1004B0000CC05695479591FD73C05695479590FD94
:1004C0006FC0D52EC42ED694C79461FD19C0AC2D33
:1004D000AC51AD2DA24008F005C0DD2089F4AC2D53
:1004E000A85C70F4A0916700A395AA2311F0A093D3
:1004F0006700AA3008F471C02092960081606DC038
:10050000A0916700AA2319F0AA95A0936700A22CD6
:100510005091BA0097FD06C0A090C800533011F466
:10052000A090D000AAEFAA0EA22DA21DCA18DA0A26
:100530004FB74170533049F4442321F087FD05C083
:10054000806803C087FF01C08F77442359F0533080
:1005500031F4AFEFC094D094CA1ADA0A03C040E075
:1005600050E020C0533049F4CC0CDD1CAAE0CA1A7C
:10057000D20818F4A0E0CA2ED22CAFEFCA16D204CB
:1005800018F04FEF50E00EC0A091AC00CA9E412D74
:10059000000C441F50E008F012C04FEF50E00FC0B5
:1005A0005695479594FF07C0552309F04FEFA42FA8
:1005B000A6954A0F521D4F3F520508F04FEF40934A
:1005C0009600816061FF09C0AFE1A095A923AB2926
:1005D0009A2F8F7DBB2009F48062A8E1A093680068
:1005E00085FF03C0AAE0A093680061FD03C085FDFC
:1005F00001C08F7E85FD03C0A6E0A0936900F8943A
:10060000A9B7A160A9BF84FF02C0A0E4ABBF3FBEF1
:10061000189511E00AC013E008C01AE006C01EE1F8
:1006200004C014E602C018EC00C005E1BB27BA956F
:10063000F1F70A95D9F71A95C1F708952AE338E733
:1006400009C020E33CE806C02AE234EB03C025E2FF
:1006500038EC00C0B091AD00BA9509F4089512E0ED
:10066000BB279798BA95F1F7919ABA95F1F79198B7
:10067000BA95F1F7979ABA95F1F7123009F0909A76
:10068000123009F4939AB091AD00BA95F1F7123097
:1006900009F09098123009F49398B7E8BA95F1F7F9
:1006A0001A95F1F6022FB22FBA95F1F70A95D9F7FC
:1006B0003A9581F697980895221B39E0001F3A95E4
:1006C00009F40895221F211B18F4210F8894F6CFF6
:1006D0000894F4CF622C722CB0E08894B395221F5A
:1006E000331FE0F7379527958894912E802E020BC3
:1006F000130B10F4192D082D10F4889401C00894E0
:10070000661C771CBA9571F7172D062D0895322DAA
:1007100011232AF43A9500951095031B130BF894B6
:10072000029F712C002D129F912C802C7894780CB4
:10073000172D921C292DB4E06B2E26951795079541
:100740006A94D9F7332321F000951095031B130BFE
:100750000895089510917B00169500917A000795F1
:10076000B0917E00B01B0B2FB0917F00B10B1B2FFF
:1007700028F40038BFEF1B0740F009C00F371205FF
:1007800008F405C00FE710E002C000E81FEF009377
:10079000830010938400089500918300B09180003D
:1007A0000B0F10918400B09181001B1F20E030914D
:1007B000840033230AF42A95B09182002B1F1AF487
:1007C000203F40F00AC02F3008F407C00FEF1FEFA2
:1007D0002FE003C000E010E020EF30916300B09103
:1007E0009B003B1718F4323030F009C0B091840000
:1007F000BB235AF004C0B0918400BB2332F40093B1
:100800008000109381002093820008952091D700EA
:1008100000918300000F10918400111F78DF1123D5
:100820002AF40038BFEF1B0740F009C00F3712054C
:1008300008F405C00FE710E002C000E81FEF002336
:1008400052F0B0916200B01B0B2F18F0013008F08D
:100850000AC001E008C000950F5FB09162000B0F65
:1008600008F001C00FEF0093850008952091D80093
:1008700000918100109182004ADF11232AF4013097
:10088000BFEF1B0740F009C00F3F120508F405C079
:100890000FEF10E002C001E01FEF112352F0B09102
:1008A0008500B01B0B2F18F0013008F00AC001E0E2
:1008B00008C000950F5FB09185000B0F08F001C0D4
:1008C0000FEF0093630008950FEF71FD1EC0B0910C
:1008D000D300BB23D1F0B0917B00BB23B1F00FEF6D
:1008E00010917B00E9DEF894B091730072FDB5E0E1
:1008F0000B9F112D002D7894112309F00FEFB0916B
:100900009E000B1710F400919E0000939D00089527
:1009100000917A0010917B0000541140B0919D002D
:1009200010F4BA9501C0B39511F0B0939D000895ED
:1009300000C008952091B500B6B1B6FDFBCF04B15B
:1009400015B1B6B1BF77B6B9B091AA00B395B0935F
:10095000AA00B83060F12092AA00B091D200BB2367
:1009600021F1112329F0B091AB00BF3F61F009C024
:10097000B091AB000B1739F020F4BB2321F0BA95EE
:1009800002C0B395E1F300919B00B093AB00B0308F
:1009900050F400ECB03038F400E8B03020F400E45B
:1009A000B03008F400E000939B007F7E0895B09182
:1009B0009B00B39511F0B0939B00B091AA00B730A3
:1009C00009F47061089502E3F894B091D9000B9F87
:1009D000012D000C001F7894B0919B000B1710F0B4
:1009E00000919B000093610000936300502E0093E0
:1009F000640000939E00089520927A00B0EFB093B7
:100A00007B000895F8940CB51DB52091740078947E
:100A10003091750060907600009375001093760019
:100A2000031B160971FD03C077FD80C028C07090BC
:100A30007700209377002709222319F00FEF1FEF8B
:100A40000EC080907800909079003093780060928A
:100A5000790000917500109176000819190920910C
:100A60007A0030917B0036952795020F131F10F402
:100A70000FEF1FEF00937A0010937B002BC02091A3
:100A80007A0030917B003901B4E08B2EB2E09B2ECE
:100A9000343040F08A949A94383020F072FD02C0CD
:100AA0008A949A94769467948A94E1F72619370980
:100AB000992021F0169507959A94E1F7200F311FA0
:100AC00020937A0030937B0028F43FEF30937A0034
:100AD00030937B00323008F4706871FF02C0B3E0DD
:100AE0000DC0B091C40000917100023838F0B39588
:100AF000003A08F0B395B63008F0B5E09B2EB4E0AC
:100B00008B2E10917B0000917A0024E016950795BA
:100B10002A95E1F70819120928F0B02FB250B12F29
:100B2000B20910F402E010E0980126C020917A008A
:100B300030917B003901769467946694669466944C
:100B40002619320906950695200F321D20937A004A
:100B500030937B00323008F07F7704E0369527959C
:100B60003695279526952695201B10F0223008F4FF
:100B700022E089019090C40060FDFECFE0908B00E0
:100B8000F0908C006160B9B7B061B9BF380177FDF2
:100B900041C07694679400938B0010938C00B92D1C
:100BA000B330E1F0B0FD04C0060D171D930106C07F
:100BB000000F111F0250120922E030E0B92DB330AE
:100BC00068F020938D0030938E000093870010937F
:100BD00088006092890070928A003AC000938D006C
:100BE00010938E00209387003093880060928900D4
:100BF00070928A0071FF0DC0BFE0B0938D0020920B
:100C00008E00B093890020928A00B0938B002092CE
:100C10008C001EC0669400938B00B92DB33091F008
:100C2000B0FD03C0060D262D03C0000F025022E0C8
:100C3000B92DB33038F020938D0000938700609277
:100C4000890006C000938D00209387006092890080
:100C500000917C0002FD0350013031F495FD0CC081
:100C6000B2E0B06CB7B90BC0023021F4B3E0B06CA5
:100C7000B7B905C095FDF4CFB4E0B06CB7B9009139
:100C8000A200000F10F4BBE60B270093A20060FD4A
:100C9000FECFB2E0B0936E006160B9B7B061B9BF8A
:100CA000B72FB670D1F020917A0030917B00369545
:100CB00027953695279571FF02C0B0E43B0FF89455
:100CC0000CB51DB5020F131F1BBD0ABD6160B0E15D
:100CD000B8BFB9B7B061B9BF789408956860209281
:100CE0007D0020E066FD20E206C0686020927D0065
:100CF00020E266FD20E001E011E077FD11C0B72F92
:100D0000B67009F0677F14E100917B00069509F445
:100D100003950F3008F00FE071FF02C004E114E109
:100D200060FD0FC0B0917D00BB2359F071FF06C07C
:100D3000B0916E00BA95B0936E0011F470624FC01E
:100D4000ABDFB0B7B77FB0BFB8B1B0B7B860B0BFB6
:100D5000B0917D00B395B0937D00B8B177FD06C02A
:100D6000B1E071FDB3E0BA95F1F7B8B1B072B21766
:100D700009F02AC071FF05C00395011708F00A9514
:100D8000CFCF63FD05C00395011708F0B4CFC8CFDE
:100D9000677FF8943CB56DB470907A00B0917B0099
:100DA000770CBB1F08F4BFEF770CBB1F08F4BFEF35
:100DB000370D6B1E6BBC3ABD6160B0E1B8BFB9B70F
:100DC000B061B9BF789497CFB0916D00B13008F49D
:100DD00092CF63FD90CF0A9509F0A2CF7F7D20913D
:100DE0008D0030918E00F894B0E1B8BF0CB51DB500
:100DF000020F131F1BBD0ABDE0908700F090880012
:100E00006160B9B7B061B9BF7894B72FB67039F0E7
:100E1000B0916D0072FFB395B0936D0009C075FF7E
:100E200007C066FD05C063FD03C0BF91BF91FAC452
:100E3000089500E063FF01C001E0F8941091710093
:100E4000B7E01B9F212D102D7894200F2695179524
:100E5000269517952695179510937100183718F455
:100E6000B8E7B093710000917100B09172000B1758
:100E700020F0606190989198939860FDFECFE0908B
:100E80008900F0908A006160B9B7B061B9BF089578
:100E9000B2E095FD0AC0F894B0937C009798959ABB
:100EA00062FF01C0939A7894F4C0F894B0937C00E8
:100EB0009798949A62FF01C0909A7894EAC0B3E040
:100EC00082FF24C095FD11C002E0F894B0937C002D
:100ED000EBE7F0E00093B1009398949862FF02C0B2
:100EE000919A01C0979A7894D4C002E0F894B09394
:100EF0007C00EBE7F0E00093B1009098959862FFDA
:100F000002C0919A01C0979A7894C3C095FD0BC016
:100F1000F894B0937C00E5E6F0E0939862FF01C09E
:100F2000919A7894B6C0F894B0937C00E5E6F0E02E
:100F3000909862FF01C0919A7894ABC0B4E095FD9F
:100F40000AC0F894B0937C009598949A62FF01C00F
:100F5000919A78949EC0F894B0937C009498959A56
:100F600062FF01C0919A789494C0B5E082FF24C0DA
:100F700095FD11C001E0F894B0937C00E1E7F0E04A
:100F80000093B1009198979862FF02C0909A01C0B7
:100F9000959A78947EC004E0F894B0937C00E5E8DC
:100FA000F0E00093B1009198979862FF02C0939A85
:100FB00001C0949A78946DC095FD0BC0F894B093DD
:100FC0007C00EFE5F0E0919862FF01C0909A789480
:100FD00060C0F894B0937C00EBE6F0E0919862FF7B
:100FE00001C0939A789455C0B6E095FD0AC0F89474
:100FF000B0937C009498979A62FF01C0909A78947D
:1010000048C0F894B0937C009598979A62FF01C00D
:10101000939A78943EC0B1E082FF24C095FD11C040
:1010200004E0F894B0937C00E5E8F0E00093B100B0
:101030009098959862FF02C0939A01C0949A789410
:1010400028C001E0F894B0937C00E1E7F0E0009361
:10105000B1009398949862FF02C0909A01C0959A4B
:10106000789417C095FD0BC0F894B0937C00EBE624
:10107000F0E0909862FF01C0939A78940AC0F894C7
:10108000B0937C00EFE5F0E0939862FF01C0909A86
:1010900078946F7E08952EE530E0F9012092B1003A
:1010A0009098919893989598979894986B7F0895B5
:1010B000A2EBB0E00FEF0D930D930D930D9303E0B2
:1010C0000D9304E00D930AE00D9301E00D9301E010
:1010D0000D9301E00D93AEEBB0E001E00D930FEF47
:1010E0000D930D930D930D930D9303E00D930FEF5F
:1010F0000D930FEF0D930D9305E20D9300ED0D93FE
:101100000AEF0D930AEF0D9304E00D930FEF0D938B
:1011100001E00D9300E00D930AE70D930FEF0D939F
:1011200000E00D9301E00D9300E00D9303E00D93BB
:1011300000E00D9308952091B9008B7FB091BA0023
:10114000B33019F09F7DB1FD90629F7BB091BB00E1
:10115000B1FD9064223011F0886001C0877F08954E
:101160000A95E00FF21DB4910895ECE1F0E00091D2
:10117000B200F6DFB093D700ECE1F0E00091B300ED
:10118000EFDFB093D800EAE2F0E00091B800E8DFCA
:10119000B093D9000091B800023008F402E0009347
:1011A0007300B091CE000FEFB23009F400EAB33013
:1011B00009F402E800937200E8E3F0E00091D50042
:1011C000CFDFB093A000089508952091C80030911A
:1011D000C900B091BA00B33009F43E5097FF02C085
:1011E00020E03FEFB32FB21B6B2EB25810F4B2E8E1
:1011F0006B2E00E00395609EB12DBD57D8F3009390
:10120000AC0008959068E1DF0ADA09DA20E030E006
:10121000B0E16B2E00DAB09196002B0F321D6A946C
:10122000C9F7B4E036952795BA95E1F7822E9F77F6
:10123000CCDF0895F894E3E0F0E0B9E0B7BFB491F3
:10124000B078C1F3F894A895B1B5B861B1BDB0E07C
:10125000B1BDB4E0BEBFBFE5BDBF1DDFB0E0B8BBF0
:10126000B0E1B7BBB0E0B5BBB0E0B4BBB0E0B2BB7F
:10127000BBEBB1BB2224A0E0B0E02D92AA31E9F78C
:10128000A0E6B0E00FEF2D920A95E9F7B1E0B09338
:10129000A2000EDF03D3B7E0B06CB7B9B6B1B4604B
:1012A000B068B6B90091CA000093AD00B1E0B09348
:1012B0006A00F894B8D9C2D9B2D9C3D9B0D9C4D9BF
:1012C000AED973D3B0D9AFD9ACD9F8940AEF1AEF2D
:1012D000A0B396FDA095A2FF1FC01A95C9F70A9565
:1012E000B1F7E0E0FCE1B591B43E39F4B591B03E20
:1012F00021F4B591BF3F09F40CC0E0E0F395F395FC
:10130000B591B83F49F4B591B43931F4B591BA3AD1
:1013100019F4EE27F69509940EDF27DF55DF55DF28
:101320000091CA000093AD00B6DEB2E0B3BFB2E0F8
:10133000BEBDB2E0B5BDB1E5B8BFB9BFB0B7B77F0C
:10134000B0BFB8B1B0B7B860B0BF63D97894F0DAC5
:1013500020927000B3E096FDB2E0B5BFB0E4BBBF31
:10136000BB27B064BABF8D7F5ED9626033E02CE0EA
:10137000B0919500BB2321F42CE03A9509F4A5CF58
:101380004ED980FFA2CF8E7FB0919600B23078F315
:10139000B92FBF710091980000939700B093980007
:1013A000B01729F72A9521F76D7FB3E096FDB2E0DB
:1013B000B5BFBB27B064BABF8D7FB091D400BB234B
:1013C00021F48062B92FB0709B2F8F7B2092670031
:1013D00028D985FF05C0B0916700BA3008F0806455
:1013E0001AD902E085FF01C000E0B0919600B01765
:1013F000B8F3F89423D922D921D9789414D920921A
:101400008600B091BA00B33009F47EC004D9B0911F
:10141000BE00B13008F478C0B0916A00B13008F471
:1014200073C085FD18C0B0919600BF3F08F46CC032
:10143000F8940DD97894F5D8B0919600B130C0F7F2
:10144000F894FCD8EAD8FAD87894EBD8B091960002
:10145000BF3FB0F3DCC2B8E09B2E9068F894B5DED5
:101460007894DFD8F8949F77B0DE80909600B091A2
:101470009600BF37789408F44FC0CBD8F894E7D8DB
:1014800078949A9451F7BEDEB82DB550B093C90048
:10149000CAD8F8948FD27894BAE09B2E9068F894CA
:1014A00094DE7894BED8F8949F778FDE8090960073
:1014B000B0919600BF37789478F7ABD8F894BED83F
:1014C000ACD8BCD878949A9449F79CDEB82DBB5F11
:1014D000B093C8000B2F1091C900125810F0100BD8
:1014E00020F4B2E80B0F0093C9009DD8F89403D202
:1014F00070D2789496D8F89468DE7894B09196007B
:10150000BF3F08F48ECF83C200919600B091860051
:101510000B1710F00093860084D801E0B091BA0058
:10152000B35009F405E0B0919600B01708F069CF08
:10153000F8948DD88CD88BD8789475D820926A007E
:1015400020926B0020926C00B0916B00B395B09329
:101550006B00BF3F71F5B0916C00B395B0936C0018
:10156000B091CC0009E1BA9559F002E3BA9541F087
:101570000DE7BA9529F00AEFBA9511F020926C00A8
:10158000B0916C00B017A8F086DD43D8B0916C0024
:10159000BA95B0936C0020926B00B091CB00B093E1
:1015A000AD00F89454D87894B091CA00B093AD00CF
:1015B00038D833D8B0916800BB2319F485FF01C037
:1015C00084CE01E085FD01C006E0B0919600B01721
:1015D00008F4BACFB091BA00B35009F022D8B09154
:1015E0006800BB2309F471CEF89455DD20926100A8
:1015F0002092620020926300522C2092640020927C
:10160000A1007894B091B700BB0FB0939F002092D7
:101610007E0020927F002092800020928100209204
:1016200082002092AA0060E070E020927100B8E091
:10163000B093AA007061EDD7B7E074FDB7E0B06C6D
:10164000B7B9B6B1B068B064B6B9B6B1B6FDFDCF42
:1016500004B115B1B6B1BF77B6B9112309F00FEFD8
:101660000093AB0067D9B8E0B093AA00706163DD66
:10167000F894BFEFB0939B00A6D9B0916100B093EE
:101680009B00B0939C00B0939D007894B1E0B09320
:101690006100B09363005B2EB0936400B093A4002C
:1016A000B0919A00B093A300B091BA00B33019F48E
:1016B0009F7D87FD90627160726020926D0094DC66
:1016C000AADC9AD99FD998D99DD996D90EDB41D851
:1016D000B0DBDEDB97D902DB65FD3CD877FFF4D8C1
:1016E00077FD16D9A6DBEBDB8DD9FFDA65FD54D883
:1016F000A0DB24DC87D9F2DA65FD88D89ADB35DCFB
:1017000081D9F3DA65FDB2D894DB6EDC7BD9E6DAF9
:10171000B7E074FDB7E0B06CB7B9B6B1B068B0640B
:10172000B6B987DB78DC6ED905D971FF21C0B091DD
:101730009E00B0939B00B0939C00B0919A00B09330
:10174000A300B1E0B093A40018E12CE0B0916D00CB
:10175000B11740F07D7F746020936F00BFEFB093AE
:101760009B0006C0B0919600B13008F0AFCF64C0C6
:1017700072FF15C066FD13C0B0916F00BA9519F4E1
:101780007B7F7860A3CFB0936F00B0919600B130AB
:1017900008F09CCFB091BA00B33009F04DC0209250
:1017A0007000B091990002E81091D600112309F061
:1017B00003E0B01708F040C085FF04C0B091680096
:1017C000BB23D1F1B091BA00B33081F495FD03C0D1
:1017D00087FD04C00BC087FF01C008C066FD06C0BE
:1017E0006064B0919E00B0939B0085CF00EF66FFD0
:1017F00005C0B0919E00B0939B0000E2B0917B00C9
:10180000B01708F463CF66FF17C06F7B9F7D87FD1D
:1018100090627460B2E1B0936F00B0919E00B0939B
:101820009B0054CFB0917000B395B0937000B0910D
:101830009600BB2309F002C020927000F8942BDCC4
:101840008090B900B2E0B093B90075DC8092B90025
:10185000209261002092620020926300522C20921C
:10186000640020929F0060E070E07894DAD613DC88
:101870000091D600002319F0909A919A939AB7E0BC
:10188000B06CB7B9B6B1B460B068B6B985FF05C081
:10189000B0917000B43008F018CD52CEEDE0F0E019
:1018A00023D00A3509F01BC0EEE0F0E01DD0053A68
:1018B00009F015C03AE0A2EBB0E0E3E0F0E014D0AC
:1018C0000D9331963A95D9F739E1AEEBB0E0EFE000
:1018D000F0E00AD00D9331963A95D9F702C0E8DBD3
:1018E0000AD0E8E2F0E00895E199FECFEEBBFFBB3D
:1018F000E09A0DB308951ED03AE0A2EBB0E0E3E029
:10190000F0E00D910FD031963A95D9F739E1AEEB71
:10191000B0E0EFE0F0E00D9105D031963A95D9F7BF
:1019200012D00895E199FECF0DBBEEBBFFBBE29A4A
:10193000E19A0895EDE0F0E00FEFF4DFEEE0F0E083
:101940000FEFF0DF0895EDE0F0E00AE5EBDFEEE009
:10195000F0E005EAE7DF08953091AE000091AF00B6
:10196000313011F40093B600323011F40093B70017
:10197000333011F40093B800343011F40093C400F4
:10198000353011F40093B900363011F40093D500CE
:10199000373011F40093CE00383011F40093BA00C0
:1019A000393011F40093BB00089525E03CD62A9508
:1019B000E9F7089543D645D647D649D62ED63ED622
:1019C00040D642D644D629D639D63BD63DD63FD688
:1019D00008953DD639D635D631D61FD638D634D629
:1019E00030D62CD61AD633D62FD62BD627D6089556
:1019F0008090AE009090AF0021D620D61FD60DD695
:101A00008A94D1F724D609D69A94E1F70895F894E8
:101A1000D1DF7894CADFC9DFB1E0B093AE00B1E0A6
:101A2000B093AF002092B000F894E2DF7894B5E074
:101A30006B2E70909600F7D5B09196007B16C9F783
:101A4000B13018F0BF3F40F107C086DFF89453DF94
:101A5000B1DFB8E0B1BDA9DF6A9459F7B091B00029
:101A6000B395B093B000B33008F4DECF9EDFB091F1
:101A7000AF00B395B093AF00F894B091AE00BA95B3
:101A8000EEE3F0E0EB0FF21D049178940395B09132
:101A9000AF00B01708F4C6CF88DF87DFB091AE0083
:101AA000B395B093AE00B091AE00BA3008F4B7CFA2
:0E1AB000FFDAF89420DFB8E0B1BD77DFBBCBE2
:00000001FF
